:1000000009C021C020C056C01EC01DC01CC01BC0DE
:100010001AC019C011241FBECFE9CDBF10E0A0E661
:10002000B0E0EAEEF2E002C005900D92A436B1070E
:10003000D9F710E0A4E6B0E001C01D92AA36B107DE
:10004000E1F751D050C1DCCFE82F409160005091D2
:100050006100609162007091630030E080E01FC039
:10006000282F220FDB01CA01B695A7959795879592
:1000700041705070607070707095609550954195AA
:100080005F4F6F4F7F4F4C7358716C7A737A48276C
:1000900059276A277B27842F8170822B3F5F3E1769
:1000A000F8F2409360005093610060936200709397
:1000B000630008951F920F920FB60F9211248F9331
:1000C000809169008150809369008F5F31F481E0F5
:1000D000809364008FE0809369008F910F900FBE32
:1000E0000F901F9018958F929F92AF92BF92CF92D0
:1000F000DF92EF92FF920F931F93CF93DF9380E0F5
:1001000090E0C9D08B019C010F5F1F4F2F4F3F4FD5
:10011000D9F3009360001093610020936200309344
:10012000630080E090E0A801B901B8D081E28FBD02
:1001300082E083BFB99A89BF7894809065009090DF
:100140006600C0916700D091680007C085B78062E3
:1001500085BF889585B78F7D85BF80916400882392
:10016000A9F31092640000E810E081E06DDF829551
:10017000807F080F1F5F1031C1F784E065DF182F03
:1001800084E062DF081B010F802F992787FD90957F
:100190006C01CC0CDD1C5601AC0EBD1E7501002798
:1001A000F7FC0095102FEC01CC0FDD1FCC0FDD1FED
:1001B000C80DD91DC801B70120E23EEF4FEF5FEF38
:1001C0002AD0672F782F892F992787FD9A95C61BEC
:1001D000D70BC801B70122EE30E040E050E01BD061
:1001E000672F782F892F992787FD9A954601861AC0
:1001F000970AC50163E970E027D065557F4F77FF07
:1002000002C060E006C06F3F710519F014F06FEF97
:1002100070E069BDA2CFFF27EE27BB27AA2760FFAA
:1002200004C0A20FB31FE41FF51F220F331F441F8A
:10023000551F969587957795679589F70097760767
:1002400071F7CF01BD01089597FB092E07260AD04B
:1002500077FD04D00CD006D000201AF4709561957B
:100260007F4F0895F6F7909581959F4F0895AA1BAB
:10027000BB1B51E107C0AA1FBB1FA617B70710F091
:10028000A61BB70B881F991F5A95A9F780959095C3
:10029000BC01CD010895A6E144E00AC0242F16D088
:1002A000252F14D000C011D0272F10C0A82F862FC3
:1002B000E82FE199FECF1FBA05C0EEBBE09AE395A7
:1002C0000DB20D924150C8F70895262FE199FECF47
:1002D0001CBA1FBA8EBB2DBB0FB6F894E29AE19AF6
:0A02E0000FBE01960895F894FFCFB9
:0402EA00010000000F
:00000001FF
